:10800000FEDF07EA000000000000000000000000A2
:108010000000000000000000000000000000000060
:108020000000000000000000000000000000000050
:108030000000000000000000000000000000000040
:108040000000000000000000000000000000000030
:02000004001FDB
:020000040020DA
:1000000002D3A0E3B80000EBFEFFFFEA001080E59A
:100010001EFF2FE1B010C0E11EFF2FE10010C0E570
:100020001EFF2FE1000090E51EFF2FE10E00A0E172
:100030001EFF2FE110FF2FE11EFF2FE110402DE9E1
:1000400008009FE5F6FFFFEB1040BDE81EFF2FE123
:100050005450212010402DE920409FE50400A0E1EC
:10006000EFFFFFEB010010E3FBFFFF0A10009FE52D
:10007000EBFFFFEB1040BDE8FF0000E21EFF2FE1A9
:10008000545021204050212010402DE90C009FE5C4
:10009000E3FFFFEB1040BDE8010000E21EFF2FE18F
:1000A0005450212070402DE90050A0E120409FE5F0
:1000B0000400A0E1DAFFFFEB200010E3FBFFFF0AE2
:1000C0000510A0E10C009FE5CFFFFFEB7040BDE8FD
:1000D0001EFF2FE1545021204050212010402DE9D7
:1000E00014409FE50400A0E1CDFFFFEB010C10E3FD
:1000F000FBFFFF1A1040BDE81EFF2FE154502120E6
:1001000070402DE90050A0E12040A0E3044044E20B
:100110003504A0E10F0000E2090050E337008082BF
:1001200030008092DEFFFFEB000054E3F6FFFF1A81
:100130002000A0E37040BDE8D9FFFFEA10402DE9A0
:10014000EEFFFFEB0D00A0E3D5FFFFEB0A00A0E3FD
:100150001040BDE8D2FFFFEA10402DE90110A0E3F6
:10016000D4009FE5A8FFFFEB0010A0E3CC009FE5C3
:10017000A5FFFFEB0010A0E3C4009FE5A2FFFFEB8B
:100180000310A0E3BC009FE59FFFFFEB0010A0E37E
:10019000B4009FE59CFFFFEB0010A0E39C009FE5EF
:1001A00099FFFFEBC610A0E3A0009FE596FFFFEBD1
:1001B0009C109FE59C009FE593FFFFEB98009FE557
:1001C00097FFFFEB3F1AC0E3121A81E388009FE517
:1001D0008DFFFFEB0010A0E380009FE58AFFFFEB9F
:1001E0000040A0E30400A0E1014084E291FFFFEBA6
:1001F000960054E3FAFFFF1A0319A0E360009FE59D
:1002000081FFFFEB0040A0E30400A0E1014084E295
:1002100088FFFFEB960054E3FAFFFF1A0010A0E3FB
:100220003C009FE578FFFFEB0310A0E310009FE583
:1002300075FFFFEB1040BDE81EFF2FE104502120A9
:1002400044502120605021204C502120505021202A
:10025000485021200E010000685021200400202079
:10026000940020209800202010402DE91C409FE59C
:10027000F918A0E30400A0E163FFFFEB0400A0E194
:100280000C109FE560FFFFEB1040BDE81EFF2FE163
:1002900008B400200002F90010402DE908009FE595
:1002A0005FFFFFEB1040BDE81EFF2FE120B40020F0
:1002B00010402DE928409FE50400A0E158FFFFEB26
:1002C0000E16C0E3021681E30400A0E14EFFFFEB2F
:1002D0000219A0E30C009FE54BFFFFEB1040BDE8C7
:1002E0001EFF2FE11000202020002020F84F2DE9D4
:1002F0000070A0E3EDFFFFEB96FFFFEB40029FE5F0
:100300008DFFFFEB48FFFFEB8BFFFFEB4900A0E306
:1003100063FFFFEB4800A0E361FFFFEB4500A0E3B4
:100320005FFFFFEB5800A0E35DFFFFEB0D00A0E3D4
:100330005BFFFFEB0A00A0E307A0A0E10760A0E1DC
:100340000750A0E10780A0E10740A0E154FFFFEBC8
:10035000F0919FE53EFFFFEB3A0050E32B00000ACF
:100360000D0050E30A00501301B0A00300B0A01329
:100370002900000A2030C0E3470053E34F00000A81
:10038000013044E2140053E303F19F97F0FFFFEACA
:1003900000042000000420009C0420009C04200095
:1003A0009C0420009C0420007C04200044042000C5
:1003B000240420002404200024042000240420001D
:1003C00018042000E4032000E4032000E4032000DC
:1003D000E4032000E4032000E4032000E403200001
:1003E000E4032000390050E3070040820AA2A0E1A4
:1003F0000F0000E2150054E30AA080E14400000A67
:1004000013FFFFEB3A0050E3014084E2D3FFFF1AF1
:100410000140A0E3CEFFFFEA0662A0E10040A0E3B6
:10042000CBFFFFEA390050E3070040820662A0E1FB
:100430000F0000E2066080E1096006E0014084E20E
:10044000C3FFFFEA390050E3070040820552A0E1F4
:100450000F0000E2055080E1FF5005E2010055E386
:100460002700000A0E40A033B9FFFF3A020055E30F
:100470000940A0030040A013B5FFFFEA390050E394
:10048000070040820552A0E10F0000E2055080E124
:10049000FF5005E20840A0E3ADFFFFEA390050E35A
:1004A000070040820882A0E10F0000E2088080E19E
:1004B000098008E0088086E1014084E2A4FFFFEAA9
:1004C0000D00A0E3F6FEFFEB2D00A0E3F4FEFFEB32
:1004D0002D00A0E3F2FEFFEB0D00A0E3F0FEFFEB2A
:1004E0000A00A0E3EEFEFFEB0A00A0E3ECFEFFEB48
:1004F0000209A0E3CEFEFFEB0B00A0E1F84FBDE840
:100500001EFF2FE10700A0E10BFFFFEB0040A0E37F
:100510008FFFFFEA6A382AE02334A0E1FF3CC3E3FF
:100520006AA423E00800A0E1077088E00A10A0E1B7
:10053000B5FEFFEB07708AE0048088E20E40A0E37E
:0C05400083FFFFEA78563412FFFF000032
:040000030000800079
:00000001FF
